:020000040000FA
:020000003028A6
:08000800F000030E8301F1007A
:100010000C180F28710E8300F00E700E0900393095
:100020008E00FC308F002208A300A303031D1A28B2
:10003000A4142928A303031D1E282928A303031D94
:1000400024281E08A5002928A303031D29289F147E
:100050002928A203031D2E281430A2000C100A2800
:10006000831203138313243085000730990083160D
:1000700051309F001B308500831264001030A800AF
:1000800030308400FF308000840A8000840A003011
:100090008000840A8000840AA803031D42281430CB
:1000A000A2000130A600303084000830A80000080B
:1000B000A90001309F0039308E00FC308F000C10F9
:1000C0000130900083160C148312C0308B00640042
:1000D000A41C67282608A700A703031D8D28A803D2
:1000E000031D7D280830A800840A70300402031D17
:1000F0007B28303084000008A9000310A90D031CE0
:1001000083288512842885162508143C031CCB28D7
:100110000230A6003230AA00CB28A703031D9C287A
:100120008516AA03031DCB2885120330A6003030A4
:1001300084000830A800CB28A703031DBA2825088F
:10014000143C031CA5288512A6288516A90DA80312
:10015000031DCB280830A80029088000840A7030CD
:100160000402031DCB28303084000430A600323056
:10017000AA00CB28A703031DCB288516AA03031DBD
:10018000CB2885120130A600303084000830A8004A
:0A0190000008A900CB28A41067287E
:00000001FF
